:100000000EC028C027C026C02CC024C023C022C0D8
:1000100021C020C01FC01EC01DC01CC01BC0112499
:100020001FBECFE5D1E0DEBFCDBF10E0A0E6B0E05F
:10003000E2E5F1E002C005900D92A036B107D9F7D4
:1000400010E0A0E6B0E001C01D92A936B107E1F7CB
:1000500004D07DC0D5CF0895089557D0FCDFFCDFD4
:10006000FECF1F920F920FB60F9211242F933F9342
:100070004F935F936F937F938F939F93AF93BF93B0
:1000800020916400309165004091660050916700B6
:1000900070916800DA01C9010296A11DB11D672F98
:1000A0006A5F6D3730F06D57DA01C9010396A11D03
:1000B000B11D609368008093640090936500A093E5
:1000C0006600B09367008091600090916100A091FC
:1000D0006200B09163000196A11DB11D8093600084
:1000E00090936100A0936200B0936300BF91AF91C1
:1000F0009F918F917F916F915F914F913F912F9140
:100100000F900FBE0F901F901895789480B780685D
:1001100080BF80B7806480BF8CB580648CBD8FEF5A
:100120008DBD80B7807F846080BF89B7846089BFC0
:1001300083B7887F83BF8AB58C7F81608ABD83B790
:10014000877F83BF83B7887F826083BF0895F894D9
:02015000FFCFDF
:00000001FF
